:10C00000B240805A200132C23D4002C23140000499
:10C01000F24080005600F2400F005700C243580023
:10C02000D2432200D2432100F24006002600F24013
:10C0300006004100F24081006100C2436000F2400E
:10C040008A006200C2436300D2C36100B240D007DD
:10C050007201B24010026001B240100062018243DE
:10C06000640132D20943B012B0C0E2B30300FD272D
:10C07000F2436700E2B30300FD27F2436700E2B337
:10C080000300FD27D24210026700E2B30300FD2740
:10C09000D2421102670037403D0008431883FE2357
:10C0A0001783FB231953DF3FE2B30300FD27304121
:10C0B0003D4004C2B012F2C0F240CC002002B012E7
:10C0C00026C1F24044002002B01226C1B0124EC177
:10C0D000B012F2C0F240CC002002B01226C1F240F1
:10C0E000BE002002B01226C1B01260C13D4002C2A3
:10C0F0003041D0C32D3FB240001E720180437240D8
:10C100000B431B93FE23D0D3193FD0C3163FD0B3AC
:10C11000103FFD23D0B30A3FFD27D0D3063FB240E6
:10C12000C00372013041F2422102D2B32002032443
:10C13000B0129AC1023CB012B6C13A4006001A834E
:10C14000FE2352112002D2832102EF2330413A40D4
:10C1500006001A83FE23B012CAC10A93F8273041A1
:10C160003E401002B24222023A4006001A83FE23E9
:10C17000B012CAC15E1100000A930424FED08000F0
:10C180000000033CFEC08000000092832202EC23EA
:10C190001E533E901902E6233041D0C3853E8043B2
:10C1A000D03F0B433A4006001A83FE23D0D3733EA0
:10C1B0001B93FE233041D0C3693E8043B43F0B4301
:10C1C0001B93FE23D0D35B3E3041D0C3553E3A4053
:10C1D00006001A83FE23D0D3493ED0C3463E804397
:10C1E000903F0B4390B33A3E01201A531B93FA231E
:10C1F000D0D3303E0A9302240A4330411A433041DF
:08C20000004D00131B43001365
:10FFE8000000000000000000000000C20000000047
:08FFF80000000000000000C041
:00000001FF
